:020000040000FA
:1000000025096600700071002F092F092F092F099B
:100010003D091106120A3106150AF007180AF00602
:100020001D0A080AF006220A080AF007220A080A2E
:10003000110506052F090604080A310506052F09D2
:100040000604080A71006600080A25000504670016
:10005000000C26000C0C0600F00C02000008020C3C
:100060003200E80C3300FF0C34000000F402350AC3
:10007000F302350AF202350A000866073D0A6607F0
:100080003F0A7000000000000000000000000000B7
:0C00900000000000B0026606420A0008F2
:021FFE00EB0FE7
:00000001FF
